 dvfc_mc34704

 Timestamp is 4da2a50f (Mon Apr 11 18:51:59 2011)

 Preferred load address is 10000000

 Start         Length     Name                   Class
 0001:00000000 00000004H .CRT$XCA                CODE
 0001:00000004 00000004H .CRT$XCZ                CODE
 0001:00000008 00000004H .CRT$XIA                CODE
 0001:0000000c 00000004H .CRT$XIZ                CODE
 0001:00000010 00000004H .CRT$XPA                CODE
 0001:00000014 00000004H .CRT$XPZ                CODE
 0001:00000018 00000004H .CRT$XTA                CODE
 0001:0000001c 00000004H .CRT$XTZ                CODE
 0001:00000020 0000099eH .rdata                  CODE
 0001:000009c0 00000029H .rdata$debug            CODE
 0001:000009ec 00002438H .text                   CODE
 0001:00002e24 00000048H .xdata                  CODE
 0001:00002e6c 00000050H .idata$2                CODE
 0001:00002ebc 00000014H .idata$3                CODE
 0001:00002ed0 000000a0H .idata$4                CODE
 0001:00002f70 000000ceH .idata$6                CODE
 0001:00003040 00000098H .edata                  CODE
 0002:00000000 000000a0H .idata$5                DATA
 0002:000000a0 00000064H .data                   DATA
 0002:00000104 0000005cH .bss                    DATA
 0003:00000000 00000180H .pdata                  DATA

  Address         Publics by Value              Rva+Base       Lib:Object

 0000:00000000       ___safe_se_handler_count   00000000     <absolute>
 0000:00000000       ___safe_se_handler_table   00000000     <absolute>
 0001:00000000       __xc_a                     10001000     corelib0:crt0init.obj
 0001:00000004       __xc_z                     10001004     corelib0:crt0init.obj
 0001:00000008       __xi_a                     10001008     corelib0:crt0init.obj
 0001:0000000c       __xi_z                     1000100c     corelib0:crt0init.obj
 0001:00000010       __xp_a                     10001010     corelib0:crt0init.obj
 0001:00000014       __xp_z                     10001014     corelib0:crt0init.obj
 0001:00000018       __xt_a                     10001018     corelib0:crt0init.obj
 0001:0000001c       __xt_z                     1000101c     corelib0:crt0init.obj
 0001:00000040       ??_C@_1EO@MKMOBHO@?$AAP?$AAm?$AAi?$AAc?$AAR?$AAe?$AAg?$AAu?$AAl?$AAa?$AAt?$AAo?$AAr?$AAG?$AAe?$AAt?$AAV?$AAo?$AAl?$AAt?$AAa?$AAg?$AAe?$AAL?$AAe?$AAv?$AAe?$AAl?$AA?5?$AAf?$AAa?$AAi@ 10001040     voltctrl.obj
 0001:00000090       ??_C@_1CG@BAGCAEII@?$AAP?$AAm?$AAi?$AAc?$AAO?$AAp?$AAe?$AAn?$AA?5?$AAf?$AAa?$AAi?$AAl?$AAe?$AAd?$AA?$CB?$AA?$AN?$AA?6?$AA?$AA@ 10001090     voltctrl.obj
 0001:000000b8       ??_C@_1CI@OHCJFJPM@?$AAE?$AAR?$AAR?$AAO?$AAR?$AA?3?$AA?5?$AA?$CF?$AAs?$AA?5?$AAl?$AAi?$AAn?$AAe?$AA?5?$AA?$CF?$AAd?$AA?3?$AA?5?$AA?$AA@ 100010b8     voltctrl.obj
 0001:000000e0       ??_C@_1KA@JKMBKCOB@?$AAc?$AA?3?$AA?2?$AAw?$AAi?$AAn?$AAc?$AAe?$AAr?$AAo?$AAo?$AAt?$AAs?$AA?2?$AAt?$AAo?$AAp?$AAa?$AAz?$AA?2?$AAw?$AAi?$AAn?$AAc?$AAe?$AA7?$AA0?$AA0?$AA?2?$AAp?$AAl?$AAa@ 100010e0     voltctrl.obj
 0001:00000180       ??_C@_1EI@DKJCDIHI@?$AAC?$AAr?$AAe?$AAa?$AAt?$AAe?$AAT?$AAh?$AAr?$AAe?$AAa?$AAd?$AA?5?$AAf?$AAa?$AAi?$AAl?$AAe?$AAd?$AA?5?$AAf?$AAo?$AAr?$AA?5?$AAD?$AAV?$AAF?$AAC?$AA?5?$AAI?$AAS?$AAT@ 10001180     dvfc_common_topaz_v1:dvfc.obj
 0001:000001c8       ??_C@_1CM@KJADCGLN@?$AAB?$AAS?$AAP?$AAD?$AAv?$AAf?$AAc?$AAI?$AAn?$AAi?$AAt?$AA?5?$AAf?$AAa?$AAi?$AAl?$AAe?$AAd?$AA?$CB?$AA?$AN?$AA?6?$AA?$AA@ 100011c8     dvfc_common_topaz_v1:dvfc.obj
 0001:000001f8       ??_C@_1FO@DKILBGK@?$AAI?$AAn?$AAt?$AAe?$AAr?$AAr?$AAu?$AAp?$AAt?$AAI?$AAn?$AAi?$AAt?$AAi?$AAa?$AAl?$AAi?$AAz?$AAe?$AA?5?$AAf?$AAa?$AAi?$AAl?$AAe?$AAd?$AA?5?$AAf?$AAo?$AAr?$AA?5?$AAD@ 100011f8     dvfc_common_topaz_v1:dvfc.obj
 0001:00000258       ??_C@_1GC@FHBKPEO@?$AAI?$AAO?$AAC?$AAT?$AAL?$AA_?$AAH?$AAA?$AAL?$AA_?$AAR?$AAE?$AAQ?$AAU?$AAE?$AAS?$AAT?$AA_?$AAS?$AAY?$AAS?$AAI?$AAN?$AAT?$AAR?$AA?5?$AAf?$AAa?$AAi?$AAl?$AAe?$AAd@ 10001258     dvfc_common_topaz_v1:dvfc.obj
 0001:000002c0       ??_C@_1FE@KIHGNMCK@?$AAC?$AAr?$AAe?$AAa?$AAt?$AAe?$AAE?$AAv?$AAe?$AAn?$AAt?$AA?5?$AAf?$AAa?$AAi?$AAl?$AAe?$AAd?$AA?5?$AAf?$AAo?$AAr?$AA?5?$AAD?$AAV?$AAF?$AAC?$AA?5?$AAI?$AAS?$AAT?$AA?5@ 100012c0     dvfc_common_topaz_v1:dvfc.obj
 0001:00000314       ??_C@_1CA@DNJNIIBE@?$AAI?$AAN?$AAT?$AAR?$AA_?$AAE?$AAV?$AAE?$AAN?$AAT?$AA_?$AAD?$AAV?$AAF?$AAC?$AA?$AA@ 10001314     dvfc_common_topaz_v1:dvfc.obj
 0001:00000334       ??_C@_1DE@BLFOHFK@?$AAR?$AAe?$AAg?$AAQ?$AAu?$AAe?$AAr?$AAy?$AAV?$AAa?$AAl?$AAu?$AAe?$AAE?$AAx?$AA?5?$AAf?$AAa?$AAi?$AAl?$AAe?$AAd?$AA?$CB?$AA?$AN?$AA?6?$AA?$AA@ 10001334     dvfc_common_topaz_v1:dvfc.obj
 0001:00000368       ??_C@_1M@EENNDIOJ@?$AAI?$AAn?$AAd?$AAe?$AAx?$AA?$AA@ 10001368     dvfc_common_topaz_v1:dvfc.obj
 0001:00000374       ??_C@_1DA@NAMEIHJM@?$AAO?$AAp?$AAe?$AAn?$AAD?$AAe?$AAv?$AAi?$AAc?$AAe?$AAK?$AAe?$AAy?$AA?5?$AAf?$AAa?$AAi?$AAl?$AAe?$AAd?$AA?$CB?$AA?$AN?$AA?6?$AA?$AA@ 10001374     dvfc_common_topaz_v1:dvfc.obj
 0001:000003a8       ??_C@_1KC@MHOHNEKI@?$AAc?$AA?3?$AA?2?$AAw?$AAi?$AAn?$AAc?$AAe?$AAr?$AAo?$AAo?$AAt?$AAs?$AA?2?$AAt?$AAo?$AAp?$AAa?$AAz?$AA?2?$AAw?$AAi?$AAn?$AAc?$AAe?$AA7?$AA0?$AA0?$AA?2?$AAp?$AAl?$AAa@ 100013a8     dvfc_common_topaz_v1:dvfc.obj
 0001:00000450       ??_C@_1EC@EEIKCCIH@?$AAU?$AAn?$AAs?$AAu?$AAp?$AAp?$AAo?$AAr?$AAt?$AAe?$AAd?$AA?5?$AAD?$AAV?$AAF?$AAC?$AA?5?$AAI?$AAO?$AAC?$AAT?$AAL?$AA?5?$AAc?$AAo?$AAd?$AAe?$AA?5?$AA?$CF?$AAu?$AA?$AN?$AA?6@ 10001450     dvfc_common_topaz_v1:dvfc.obj
 0001:00000498       ??_C@_1EI@MGFJEBDP@?$AAE?$AAx?$AAc?$AAe?$AAp?$AAt?$AAi?$AAo?$AAn?$AA?5?$AAi?$AAn?$AA?5?$AAD?$AAV?$AAF?$AAC?$AA?5?$AAI?$AAO?$AAC?$AAT?$AAL?$AA_?$AAP?$AAO?$AAW?$AAE?$AAR?$AA_?$AAS?$AAE@ 10001498     dvfc_common_topaz_v1:dvfc.obj
 0001:000004e0       ??_C@_1FK@CFOKMKHC@?$AAE?$AAx?$AAc?$AAe?$AAp?$AAt?$AAi?$AAo?$AAn?$AA?5?$AAi?$AAn?$AA?5?$AAD?$AAV?$AAF?$AAC?$AA?5?$AAI?$AAO?$AAC?$AAT?$AAL?$AA_?$AAP?$AAO?$AAW?$AAE?$AAR?$AA_?$AAC?$AAA@ 100014e0     dvfc_common_topaz_v1:dvfc.obj
 0001:0000053c       ??_C@_1DE@PEIHFJNG@?$AAB?$AAS?$AAP?$AAD?$AAv?$AAf?$AAc?$AAP?$AAo?$AAw?$AAe?$AAr?$AAS?$AAe?$AAt?$AA?5?$AAf?$AAa?$AAi?$AAl?$AAe?$AAd?$AA?$CB?$AA?$AN?$AA?6?$AA?$AA@ 1000153c     dvfc:dvfc.obj
 0001:00000570       ??_C@_1EE@OFPACOHL@?$AAD?$AAv?$AAf?$AAc?$AAI?$AAn?$AAi?$AAt?$AAV?$AAo?$AAl?$AAt?$AAa?$AAg?$AAe?$AAS?$AAu?$AAp?$AAp?$AAl?$AAi?$AAe?$AAs?$AA?5?$AAf?$AAa?$AAi?$AAl?$AAe?$AAd?$AA?$CB?$AA?$AN@ 10001570     dvfc:dvfc.obj
 0001:000005b8       ??_C@_1FM@FLIAFKCL@?$AAC?$AAr?$AAe?$AAa?$AAt?$AAe?$AAT?$AAh?$AAr?$AAe?$AAa?$AAd?$AA?5?$AAf?$AAa?$AAi?$AAl?$AAe?$AAd?$AA?5?$AAf?$AAo?$AAr?$AA?5?$AAD?$AAV?$AAF?$AAC?$AA?5?$AAw?$AAo?$AAr@ 100015b8     dvfc:dvfc.obj
 0001:00000614       ??_C@_1CE@KCPPCGKP@?$AAE?$AAV?$AAE?$AAN?$AAT?$AA_?$AAD?$AAV?$AAF?$AAC?$AA_?$AAW?$AAO?$AAR?$AAK?$AAE?$AAR?$AA?$AA@ 10001614     dvfc:dvfc.obj
 0001:00000638       ??_C@_1CM@PPPGIKAO@?$AAC?$AAr?$AAe?$AAa?$AAt?$AAe?$AAE?$AAv?$AAe?$AAn?$AAt?$AA?5?$AAf?$AAa?$AAi?$AAl?$AAe?$AAd?$AA?$CB?$AA?$AN?$AA?6?$AA?$AA@ 10001638     dvfc:dvfc.obj
 0001:00000664       ??_C@_1BO@ICEODACO@?$AAE?$AAV?$AAE?$AAN?$AAT?$AA_?$AAS?$AAE?$AAT?$AAP?$AAO?$AAI?$AAN?$AAT?$AA?$AA@ 10001664     dvfc:dvfc.obj
 0001:00000684       ??_C@_1CO@FMOECGMA@?$AAM?$AAm?$AAM?$AAa?$AAp?$AAI?$AAo?$AAS?$AAp?$AAa?$AAc?$AAe?$AA?5?$AAf?$AAa?$AAi?$AAl?$AAe?$AAd?$AA?$CB?$AA?$AN?$AA?6?$AA?$AA@ 10001684     dvfc:dvfc.obj
 0001:000006b8       ??_C@_1JG@EGMIOBNL@?$AAc?$AA?3?$AA?2?$AAw?$AAi?$AAn?$AAc?$AAe?$AAr?$AAo?$AAo?$AAt?$AAs?$AA?2?$AAt?$AAo?$AAp?$AAa?$AAz?$AA?2?$AAw?$AAi?$AAn?$AAc?$AAe?$AA7?$AA0?$AA0?$AA?2?$AAp?$AAl?$AAa@ 100016b8     dvfc:dvfc.obj
 0001:00000750       ??_C@_1M@LCEEOPDH@?$AAI?$AA2?$AAC?$AA1?$AA?3?$AA?$AA@ 10001750     pmicsdk:mc34704sdk.obj
 0001:0000075c       ??_C@_1DC@HNHAGOEA@?$AA?5?$AAR?$AAe?$AAg?$AAu?$AAl?$AAa?$AAt?$AAo?$AAr?$AA?5?$AAn?$AAo?$AAt?$AA?5?$AAs?$AAu?$AAp?$AAp?$AAo?$AAr?$AAt?$AAe?$AAd?$AA?$AA@ 1000175c     pmicsdk:mc34704sdk.obj
 0001:00000790       ??_C@_1EO@LPFNDCLA@?$AAR?$AAe?$AAg?$AAu?$AAl?$AAa?$AAt?$AAo?$AAr?$AA?5?$AA8?$AA?5?$AAm?$AAa?$AAn?$AAa?$AAg?$AAe?$AAm?$AAe?$AAn?$AAt?$AA?5?$AAn?$AAo?$AAt?$AA?5?$AAi?$AAm?$AAp?$AAl?$AAe@ 10001790     pmicsdk:mc34704sdk.obj
 0001:000007e0       ??_C@_1EO@KLNCGMFD@?$AAR?$AAe?$AAg?$AAu?$AAl?$AAa?$AAt?$AAo?$AAr?$AA?5?$AA7?$AA?5?$AAm?$AAa?$AAn?$AAa?$AAg?$AAe?$AAm?$AAe?$AAn?$AAt?$AA?5?$AAn?$AAo?$AAt?$AA?5?$AAi?$AAm?$AAp?$AAl?$AAe@ 100017e0     pmicsdk:mc34704sdk.obj
 0001:00000830       ??_C@_1EO@OBBFGDMA@?$AAR?$AAe?$AAg?$AAu?$AAl?$AAa?$AAt?$AAo?$AAr?$AA?5?$AA6?$AA?5?$AAm?$AAa?$AAn?$AAa?$AAg?$AAe?$AAm?$AAe?$AAn?$AAt?$AA?5?$AAn?$AAo?$AAt?$AA?5?$AAi?$AAm?$AAp?$AAl?$AAe@ 10001830     pmicsdk:mc34704sdk.obj
 0001:00000880       ??_C@_1EO@DOFMHDHF@?$AAR?$AAe?$AAg?$AAu?$AAl?$AAa?$AAt?$AAo?$AAr?$AA?5?$AA5?$AA?5?$AAm?$AAa?$AAn?$AAa?$AAg?$AAe?$AAm?$AAe?$AAn?$AAt?$AA?5?$AAn?$AAo?$AAt?$AA?5?$AAi?$AAm?$AAp?$AAl?$AAe@ 10001880     pmicsdk:mc34704sdk.obj
 0001:000008d0       ??_C@_1EO@HEJLHMOG@?$AAR?$AAe?$AAg?$AAu?$AAl?$AAa?$AAt?$AAo?$AAr?$AA?5?$AA4?$AA?5?$AAm?$AAa?$AAn?$AAa?$AAg?$AAe?$AAm?$AAe?$AAn?$AAt?$AA?5?$AAn?$AAo?$AAt?$AA?5?$AAi?$AAm?$AAp?$AAl?$AAe@ 100018d0     pmicsdk:mc34704sdk.obj
 0001:00000920       ??_C@_1EO@BBHIFLMN@?$AAR?$AAe?$AAg?$AAu?$AAl?$AAa?$AAt?$AAo?$AAr?$AA?5?$AA2?$AA?5?$AAm?$AAa?$AAn?$AAa?$AAg?$AAe?$AAm?$AAe?$AAn?$AAt?$AA?5?$AAn?$AAo?$AAt?$AA?5?$AAi?$AAm?$AAp?$AAl?$AAe@ 10001920     pmicsdk:mc34704sdk.obj
 0001:00000970       ??_C@_1EO@MODBELHI@?$AAR?$AAe?$AAg?$AAu?$AAl?$AAa?$AAt?$AAo?$AAr?$AA?5?$AA1?$AA?5?$AAm?$AAa?$AAn?$AAa?$AAg?$AAe?$AAm?$AAe?$AAn?$AAt?$AA?5?$AAn?$AAo?$AAt?$AA?5?$AAi?$AAm?$AAp?$AAl?$AAe@ 10001970     pmicsdk:mc34704sdk.obj
 0001:000009ec       DvfcInitVoltageSupplies    100019ec f   voltctrl.obj
 0001:00000acc       DvfcConvertVoltage         10001acc f   voltctrl.obj
 0001:00000bec       DvfcUpdateSupplyVoltage    10001bec f   voltctrl.obj
 0001:00000d7c       DllEntry                   10001d7c f   dvfc_common_topaz_v1:dvfc.obj
 0001:00000db8       DVF_Init                   10001db8 f   dvfc_common_topaz_v1:dvfc.obj
 0001:000010d0       DVF_Deinit                 100020d0 f   dvfc_common_topaz_v1:dvfc.obj
 0001:000010fc       DVF_Open                   100020fc f   dvfc_common_topaz_v1:dvfc.obj
 0001:00001120       DVF_Close                  10002120 f   dvfc_common_topaz_v1:dvfc.obj
 0001:0000114c       DVF_IOControl              1000214c f   dvfc_common_topaz_v1:dvfc.obj
 0001:00001488       GetCurrentThread           10002488 f i dvfc_common_topaz_v1:dvfc.obj
 0001:000014a0       BSPDvfcGetThreadPriority   100024a0 f   dvfc:dvfc.obj
 0001:000014c0       DvfcMapDevPwrStateToSetpoint 100024c0 f   dvfc:dvfc.obj
 0001:00001558       BSPDvfcGetSupportedDx      10002558 f   dvfc:dvfc.obj
 0001:00001570       BSPDvfcPowerGet            10002570 f   dvfc:dvfc.obj
 0001:000015e0       BSPDvfcPowerSet            100025e0 f   dvfc:dvfc.obj
 0001:000016f4       DvfcUpdateSetpoint         100026f4 f   dvfc:dvfc.obj
 0001:0000184c       BSPDvfcIntrServ            1000284c f   dvfc:dvfc.obj
 0001:00001898       BSPDvfcInit                10002898 f   dvfc:dvfc.obj
 0001:00001f38       BSPDvfcDeinit              10002f38 f   dvfc:dvfc.obj
 0001:00001f50       SetEvent                   10002f50 f i dvfc:dvfc.obj
 0001:00001f84       NKDbgPrintfW               10002f84 f   coredll:COREDLL.dll
 0001:00001f94       DisableThreadLibraryCalls  10002f94 f   coredll:COREDLL.dll
 0001:00001fa4       CreateThread               10002fa4 f   coredll:COREDLL.dll
 0001:00001fb4       InterruptInitialize        10002fb4 f   coredll:COREDLL.dll
 0001:00001fc4       KernelIoControl            10002fc4 f   coredll:COREDLL.dll
 0001:00001fd4       CreateEventW               10002fd4 f   coredll:COREDLL.dll
 0001:00001fe4       RegCloseKey                10002fe4 f   coredll:COREDLL.dll
 0001:00001ff4       RegQueryValueExW           10002ff4 f   coredll:COREDLL.dll
 0001:00002004       OpenDeviceKey              10003004 f   coredll:COREDLL.dll
 0001:00002014       SetLastError               10003014 f   coredll:COREDLL.dll
 0001:00002024       InterruptDone              10003024 f   coredll:COREDLL.dll
 0001:00002034       WaitForSingleObject        10003034 f   coredll:COREDLL.dll
 0001:00002044       CeSetThreadPriority        10003044 f   coredll:COREDLL.dll
 0001:00002054       QueryPerformanceFrequency  10003054 f   coredll:COREDLL.dll
 0001:00002064       QueryPerformanceCounter    10003064 f   coredll:COREDLL.dll
 0001:00002074       EventModify                10003074 f   coredll:COREDLL.dll
 0001:00002084       MmMapIoSpace               10003084 f   ceddk:CEDDK.dll
 0001:00002094       DDKClockSetpointRequest    10003094 f   cspddk:CSPDDK.dll
 0001:000020a4       DDKClockSetpointRelease    100030a4 f   cspddk:CSPDDK.dll
 0001:000020b4       DDKClockGetSharedConfig    100030b4 f   cspddk:CSPDDK.dll
 0001:000020c4       DDKClockUnlock             100030c4 f   cspddk:CSPDDK.dll
 0001:000020d4       DDKClockLock               100030d4 f   cspddk:CSPDDK.dll
 0001:000020e4       PmicOpen                   100030e4 f   pmicsdk:mc34704sdk.obj
 0001:00002158       PmicClose                  10003158 f   pmicsdk:mc34704sdk.obj
 0001:00002180       PmicEnable                 10003180 f   pmicsdk:mc34704sdk.obj
 0001:000021c4       PmicRegulatorSetVoltageLevel 100031c4 f   pmicsdk:mc34704sdk.obj
 0001:00002334       PmicRegulatorGetVoltageLevel 10003334 f   pmicsdk:mc34704sdk.obj
 0001:000024c0       PmicSetRegister            100034c0 f   pmicsdk:mc34704sdk.obj
 0001:000025ac       PmicGetRegister            100035ac f   pmicsdk:mc34704sdk.obj
 0001:0000267c       DllMain                    1000367c f   corelib0:dllmain.obj
 0001:000026b4       _DllMainCRTStartup         100036b4 f   corelib0:pegdmain.obj
 0001:0000284c       __security_init_cookie     1000384c f   corelib0:seccinit.obj
 0001:000028e4       exit                       100038e4 f   corelib0:cexit.obj
 0001:00002a08       _exit                      10003a08 f   corelib0:cexit.obj
 0001:00002a28       _cexit                     10003a28 f   corelib0:cexit.obj
 0001:00002a40       _c_exit                    10003a40 f   corelib0:cexit.obj
 0001:00002a58       _initterm                  10003a58 f   corelib0:crt0dat.obj
 0001:00002aa4       _cinit                     10003aa4 f   corelib0:crt0dat.obj
 0001:00002ad4       __crt_ExitProcess          10003ad4 f   corelib0:exitproc_proxy.obj
 0001:00002b00       GetCurrentProcess          10003b00 f i corelib0:exitproc_proxy.obj
 0001:00002b18       _onexit                    10003b18 f   corelib0:onexit.obj
 0001:00002cf4       atexit                     10003cf4 f   corelib0:onexit.obj
 0001:00002d44       memset                     10003d44 f   corelib1:COREDLL.dll
 0001:00002d54       __C_specific_handler       10003d54 f   corelib1:COREDLL.dll
 0001:00002d64       __rt_sdiv64by64            10003d64 f   corelib1:COREDLL.dll
 0001:00002d74       _XcptFilter                10003d74 f   corelib1:COREDLL.dll
 0001:00002d84       __security_gen_cookie2     10003d84 f   corelib1:COREDLL.dll
 0001:00002d94       free                       10003d94 f   corelib1:COREDLL.dll
 0001:00002da4       realloc                    10003da4 f   corelib1:COREDLL.dll
 0001:00002db4       malloc                     10003db4 f   corelib1:COREDLL.dll
 0001:00002dc4       _msize                     10003dc4 f   corelib1:COREDLL.dll
 0001:00002dd4       CloseHandle                10003dd4 f   coredll:COREDLL.dll
 0001:00002de4       TerminateProcess           10003de4 f   coredll:COREDLL.dll
 0001:00002df4       I2COpenHandle              10003df4 f   i2csdk:I2CSDK.dll
 0001:00002e04       I2CTransfer                10003e04 f   i2csdk:I2CSDK.dll
 0001:00002e14       I2CSetFrequency            10003e14 f   i2csdk:I2CSDK.dll
 0001:00002e6c       __IMPORT_DESCRIPTOR_COREDLL 10003e6c     coredll:COREDLL.dll
 0001:00002e80       __IMPORT_DESCRIPTOR_CEDDK  10003e80     ceddk:CEDDK.dll
 0001:00002e94       __IMPORT_DESCRIPTOR_CSPDDK 10003e94     cspddk:CSPDDK.dll
 0001:00002ea8       __IMPORT_DESCRIPTOR_I2CSDK 10003ea8     i2csdk:I2CSDK.dll
 0001:00002ebc       __NULL_IMPORT_DESCRIPTOR   10003ebc     coredll:COREDLL.dll
 0002:00000000       __imp_MmMapIoSpace         10005000     ceddk:CEDDK.dll
 0002:00000004       \177CEDDK_NULL_THUNK_DATA  10005004     ceddk:CEDDK.dll
 0002:00000008       __imp_CreateThread         10005008     coredll:COREDLL.dll
 0002:0000000c       __imp_InterruptInitialize  1000500c     coredll:COREDLL.dll
 0002:00000010       __imp_KernelIoControl      10005010     coredll:COREDLL.dll
 0002:00000014       __imp_CreateEventW         10005014     coredll:COREDLL.dll
 0002:00000018       __imp_RegCloseKey          10005018     coredll:COREDLL.dll
 0002:0000001c       __imp_RegQueryValueExW     1000501c     coredll:COREDLL.dll
 0002:00000020       __imp_OpenDeviceKey        10005020     coredll:COREDLL.dll
 0002:00000024       __imp_DisableThreadLibraryCalls 10005024     coredll:COREDLL.dll
 0002:00000028       __imp_InterruptDone        10005028     coredll:COREDLL.dll
 0002:0000002c       __imp_WaitForSingleObject  1000502c     coredll:COREDLL.dll
 0002:00000030       __imp_CeSetThreadPriority  10005030     coredll:COREDLL.dll
 0002:00000034       __imp_QueryPerformanceFrequency 10005034     coredll:COREDLL.dll
 0002:00000038       __imp_QueryPerformanceCounter 10005038     coredll:COREDLL.dll
 0002:0000003c       __imp_EventModify          1000503c     coredll:COREDLL.dll
 0002:00000040       __imp_SetLastError         10005040     coredll:COREDLL.dll
 0002:00000044       __imp_NKDbgPrintfW         10005044     coredll:COREDLL.dll
 0002:00000048       __imp_CloseHandle          10005048     coredll:COREDLL.dll
 0002:0000004c       __imp__msize               1000504c     corelib1:COREDLL.dll
 0002:00000050       __imp_malloc               10005050     corelib1:COREDLL.dll
 0002:00000054       __imp_realloc              10005054     corelib1:COREDLL.dll
 0002:00000058       __imp_free                 10005058     corelib1:COREDLL.dll
 0002:0000005c       __imp___security_gen_cookie2 1000505c     corelib1:COREDLL.dll
 0002:00000060       __imp_memset               10005060     corelib1:COREDLL.dll
 0002:00000064       __imp___C_specific_handler 10005064     corelib1:COREDLL.dll
 0002:00000068       __imp___rt_sdiv64by64      10005068     corelib1:COREDLL.dll
 0002:0000006c       __imp__XcptFilter          1000506c     corelib1:COREDLL.dll
 0002:00000070       __imp_TerminateProcess     10005070     coredll:COREDLL.dll
 0002:00000074       \177COREDLL_NULL_THUNK_DATA 10005074     coredll:COREDLL.dll
 0002:00000078       __imp_DDKClockUnlock       10005078     cspddk:CSPDDK.dll
 0002:0000007c       __imp_DDKClockGetSharedConfig 1000507c     cspddk:CSPDDK.dll
 0002:00000080       __imp_DDKClockSetpointRelease 10005080     cspddk:CSPDDK.dll
 0002:00000084       __imp_DDKClockSetpointRequest 10005084     cspddk:CSPDDK.dll
 0002:00000088       __imp_DDKClockLock         10005088     cspddk:CSPDDK.dll
 0002:0000008c       \177CSPDDK_NULL_THUNK_DATA 1000508c     cspddk:CSPDDK.dll
 0002:00000090       __imp_I2CTransfer          10005090     i2csdk:I2CSDK.dll
 0002:00000094       __imp_I2CSetFrequency      10005094     i2csdk:I2CSDK.dll
 0002:00000098       __imp_I2COpenHandle        10005098     i2csdk:I2CSDK.dll
 0002:0000009c       \177I2CSDK_NULL_THUNK_DATA 1000509c     i2csdk:I2CSDK.dll
 0002:000000a0       g_DvfcIrq                  100050a0     dvfc:dvfc.obj
 0002:000000fc       __security_cookie          100050fc     corelib0:seccinit.obj
 0002:00000100       __security_cookie_complement 10005100     corelib0:seccinit.obj
 0002:0000014c       _exitflag                  1000514c     corelib0:cexit.obj
 0002:00000150       g_pCRM                     10005150     <common>
 0002:00000154       __onexitend                10005154     <common>
 0002:00000158       __onexitbegin              10005158     <common>
 0002:0000015c       _pRawDllMain               1000515c     <common>

 entry point at        0001:000026b4

 Static symbols

 0001:000013f4       DvfcIntrServThread         100023f4 f   dvfc_common_topaz_v1:dvfc.obj
 0001:00001b74       DvfcWorkerThread           10002b74 f   dvfc:dvfc.obj
 0001:00002704       _DllMainCRTStartupHelper   10003704 f   corelib0:pegdmain.obj
 0001:00002904       doexit                     10003904 f   corelib0:cexit.obj
